:1000000012C02CC02BC02AC029C028C027C026C0BF
:1000100025C025C023C022C021C020C0BEC11EC033
:100020001DC01CC01BC011241FBECFE5D4E0DEBF25
:10003000CDBF11E0A0E6B0E0EEE2F9E102C005902C
:100040000D92AE3BB107D9F712E0AEEBB1E001C0C3
:100050001D92A934B107E1F72CD467CCCFC01F9211
:100060000F920FB60F9211242F938F939F93AF93FC
:10007000BF938091C0019091C101A091C201B09144
:10008000C3010196A11DB11D8093C0019093C101D0
:10009000A093C201B093C30128EF22BF80569A4EAD
:1000A000A040B040D8F08091C4019091C501A091CA
:1000B000C601B091C7010196A11DB11D8093C40175
:1000C0009093C501A093C601B093C7011092C001DF
:1000D0001092C1011092C2011092C301BF91AF9161
:1000E0009F918F912F910F900FBE0F901F90189599
:1000F000EF92FF920F931F93CF93DF93EC017B015D
:10010000D901888199818217930720F0FB016081D2
:1001100071816BC0CA010197BC01660F771FFE0198
:10012000E60FF71F808191812817390730F0F7011A
:10013000E60FF71F6081718158C0415000E01FC079
:10014000C901860F971F95958795282F90E0BC01D0
:10015000660F771FFE01E60FF71F0190F081E02D7B
:10016000AE17BF0710F4422F0AC0EA17FB0730F0A2
:10017000F701E60FF71F6081718137C0022F602FF2
:1001800070E0242F30E0CB01019682179307C4F270
:10019000A901440F551FCB01880F991FF701E80FE4
:1001A000F91F00811181F701E40FF51F20813181D2
:1001B000201B310BFE01E80FF91F80819181A81BE4
:1001C000B90BFE01E40FF51F60817181681B790B8B
:1001D000A29FC001A39F900DB29F900D11247ADBC6
:1001E000862F972FBC01600F711F862F972FDF91ED
:1001F000CF911F910F91FF90EF90089518952F9236
:100200003F924F925F926F927F928F929F92AF92A6
:10021000BF92CF92DF92EF92FF920F931F932B0129
:100220003C01F22ED32E302E212E0F2EFAE48F2EEB
:10023000F1E09F2EF02DF4011082C401BA015EDBC3
:10024000EF2DFD2DDF010D900020E9F71197AE1B7A
:10025000BF0BC4016F2D7D2DAD0157DB0F2EF6E3D3
:10026000AF2EF2E0BF2EF02DC301B2014E2D2C2D8A
:100270008501F2D7F50101900020E9F73197EA19DD
:10028000FB09C401B501AF0140DBE32DF22DDF0115
:100290000D900020E9F71197AE1BBF0BC401632D31
:1002A000722DAD0132DB1F910F91FF90EF90DF9027
:1002B000CF90BF90AF909F908F907F906F905F9006
:1002C0004F903F902F900895FF920F931F93CF93DD
:1002D000DF93F82EC82FD0E0FE01EE0FFF1FEC0FCA
:1002E000FD1FEE0FFF1FEE0FFF1FEE0FFF1FE2536C
:1002F000FE4F9F01205F3F4FD9014D915D916D9160
:100300007C91448B558B668B778B84859585A685F0
:10031000B785F90180839183A283B383FF20E1F441
:1003200084B195B1B2D58E01000F111F0C0F1D1FA6
:10033000000F111F000F111F000F111F06521E4F3B
:1003400020E030E040E251E413D9D8016D937D9371
:100350008D939C93139714C084B195B196D5FE01EB
:10036000EE0FFF1FEC0FFD1FEE0FFF1FEE0FFF1F25
:10037000EE0FFF1FE652FE4F6083718382839383EB
:1003800088E1F89EC001112482539E4F7BD4DF91F7
:10039000CF911F910F91FF9008951F920F920FB66A
:1003A0000F9211242F933F934F935F936F937F93FB
:1003B0008F939F93AF93BF93EF93FF938091BE0171
:1003C0009091BF0101969093BF018093BE01843646
:1003D000910548F483E078DFE7E2F0E08081807FF8
:1003E000856080831CC0883C910548F482E06CDF06
:1003F000E7E2F0E08081807F8460808310C08C52CF
:10040000914048F480E060DFE7E2F0E08081807FA7
:100410008360808304C01092BF011092BE01E6E2A7
:10042000F0E08081886480837894FF91EF91BF91A0
:10043000AF919F918F917F916F915F914F913F917C
:100440002F910F900FBE0F901F901895CF92DF92B3
:10045000EF92FF920F931F9380916401823059F0C5
:10046000833019F0813099F40CC08EE060E040E6F2
:1004700050E021D611C08EE060E043E650E01BD68C
:100480000BC08EE060E046E650E015D605C08EE079
:1004900060E049E650E00FD60F2EF6E1CF2EF2E0F5
:1004A000DF2EF02DF60160817181828193810F2E04
:1004B000F5E6EF2EF1E0FF2EF02D44E021E087017C
:1004C000CBD682E060E0A701F6D588EE9FEFC80E9C
:1004D000D91EF601608171818281938144E021E01F
:1004E000BBD682E061E0A701E6D56091CE017091B4
:1004F000CF018091D0019091D10143E021E0ACD6B1
:1005000087E060E0A701D7D56091630170E080E0EB
:1005100090E0C7D842E020E09FD688E061E0A701E4
:10052000CAD56091C4017091C5018091C6019091B6
:10053000C701B7D843E020E08FD68BE060E0A70189
:10054000BAD5F601608171818281938120E030E02B
:1005500040E251E45CD979D88B019C018AE891E0B2
:100560006EE971E04AE050E09801C2DD8093C80175
:1005700090E0A0E0B0E0BC01CD0193D843E020E0E2
:1005800087016AD68DE061E0A70195D51F910F9193
:10059000FF90EF90DF90CF9008952F923F924F926F
:1005A0005F926F927F928F929F92AF92BF92CF9203
:1005B000DF92EF92FF920F931F93CF93DF931092EE
:1005C000CB011092CA011092CD011092CC010F2ED6
:1005D000FEEF2F2EF1E03F2EF02DC2E3D0E00F2EE4
:1005E000F0E24F2EFEE45F2EF02DF101A080B180ED
:1005F000C280D380E0906A01F0906B0100916C01A1
:1006000010916D01C601B501A8019701ADD78823EE
:1006100054F5E0924002F09241020093420210939E
:100620004302F3E0F093640122E02093630110920F
:10063000480221E08881877F88838881846088835D
:10064000C2010197F1F788818860888388818B7F58
:100650008883C2010197F1F72F5F2B3059F78AE0A9
:1006600080934802C5C060906E0170906F018090C9
:10067000700190907101C601B501A401930174D776
:1006800088230CF04BC0C601B501A8019701BBD867
:1006900088230CF443C06092400270924102809221
:1006A000420290924302E1E0E0936401F101608133
:1006B000718182819381A401930156D788239CF490
:1006C000EEECF1E0608171818281938120E030E085
:1006D00040E450E449D7181634F0809163018F5FED
:1006E0008093630105C08091630181508093630111
:1006F0001092480220E0888188608883C2010197B7
:10070000F1F78881877F8883C2010197F1F72F5F16
:100710002A3089F7FAE0F09348026AC0C601B501B1
:10072000A401930170D818161CF02FEF3FEFACC056
:1007300020917201309173014091740150917501C3
:10074000822F932FA42FB52F8093400290934102C4
:10075000A0934202B093430282E080936401F101CE
:10076000E080F18002811381D22EC32EB42EA52EFB
:10077000C801B70148D8181634F48091630181503C
:100780008093630105C0809163018F5F8093630153
:1007900080916301853018F4F5E0F093630120E067
:1007A000888184608883C2010197F1F788818B7FFB
:1007B0008883C2010197F1F72F5F2A3089F72093D0
:1007C0004802C801B7012D2D3C2D4B2D5A2D1BD8A9
:1007D000882374F0EEECF1E0608171818281938175
:1007E0002AE939E949E95EE3BFD618160CF04AC098
:1007F0002091CC013091CD012530310538F0809128
:100800006401833019F421E030E03EC02930310525
:1008100038F080916401813019F422E030E034C076
:100820002530310538F080916401823019F423E0DD
:1008300030E02AC080916301813620F0F0E6F09329
:10084000630105C0853018F425E020936301809191
:100850006301F9D1FBDD8091CA019091CB01019632
:100860009093CB018093CA0181569A4E08F4BDCE75
:100870008091CC019091CD0101969093CD01809310
:10088000CC01B3CE20E030E0822F932FDF91CF91C7
:100890001F910F91FF90EF90DF90CF90BF90AF909E
:1008A0009F908F907F906F905F904F903F902F9090
:1008B00008952F923F924F925F926F927F928F9204
:1008C0009F92AF92BF92CF92DF92EF92FF920F93DF
:1008D0001F93CF93DF9385E083BF88EF82BFE9E565
:1008E000F0E08081816080838FEF87BBE8E3F0E0F8
:1008F000808380818D7F8083BAD180E0A4D1789479
:100900008BD311D4E4E3F0E0808187608083E1E35E
:10091000F0E080818C6F8083E2E3F0E0808188608A
:10092000808380818460808380E060E04CE650E0DA
:10093000C2D380E061E044EF50E0BDD321E0E2E3C8
:10094000F0E040E45CE98081877F8083808184607F
:100950008083CA010197F1F780818860808380815C
:100960008B7F8083CA010197F1F72F5F233359F7FB
:1009700082E380934802D7D380E060E044EF50E008
:100980009AD380E061E04DE750E095D380E061E0EC
:100990004EE850E090D36091FE017091FF0180918C
:1009A0000002909101020F2EF5E6EF2EF1E0FF2EEE
:1009B000F02D44E021E087014FD482E061E0A701FF
:1009C0007AD31092480221E3E2E3F0E040E25EE4F1
:1009D0008081877F8083808184608083CA010197C2
:1009E000F1F780818860808380818B7F8083CA015A
:1009F0000197F1F7215060F782E3809348020F2EB0
:100A0000F6E12F2EF2E03F2EF02D0F2EF4EF6F2E99
:100A1000F0E07F2EF02D0F2EF5E68F2EF1E09F2EC9
:100A2000F02D0F2EFEEF4F2EF1E05F2EF02DC8ECD3
:100A3000D0E0F101E080F18002811381C801B701AB
:100A40002DEC3CEC4CE651E48FD58823BCF480E0DF
:100A500060E0A30130D380E061E041E950E02BD3B6
:100A6000F101608171818281938144E021E0840100
:100A7000F3D38CE061E0A4011ED3DBCFF201A080B0
:100A8000B180C280D380C601B50120E030E040EAE9
:100A900050E46AD58823D4F480E060E0A3010BD34E
:100AA00080E061E042EA50E006D3F20160817181AA
:100AB0008281938144E021E08401CED38CE061E027
:100AC000A401F9D2BAD01092C801B3CF8091C80165
:100AD000882309F046C0B7D080E060E0A301EBD2E4
:100AE00080E061E044EB50E0E6D220E137E2CE0165
:100AF0000197F1F721503040D1F7F2016081718107
:100B00008281938120E030E040E251E480D69DD59F
:100B10008B019C018AE891E06EE971E04AE050E0C7
:100B20009801E6DA8093C80190E0A0E0B0E0BC0153
:100B3000CD01B7D543E020E084018ED380E061E0B1
:100B400045EC50E0B8D28DE061E0A401B4D228E8D1
:100B500033E1CE010197F1F721503040D1F75DD05C
:100B600068CFC801B7012DEC3CEC4CE651E44BD604
:100B700018160CF048C0C601B50120916A013091E9
:100B80006B0140916C0150916D013DD61816DCF55A
:100B900080916E0190916F01A0917001B0917101EF
:100BA0008093400290934102A0934202B09343028B
:100BB00085E049D080E060E046ED50E07CD280E006
:100BC00061E049ED50E077D28AE060E04CED50E022
:100BD00072D286E061E04EED50E06DD28AE061E0D5
:100BE00041EE50E068D26091630170E080E090E0F7
:100BF00058D542E020E084012FD388E061E0A401D1
:100C00005AD2CBDC16CF80E060E0A30154D280E062
:100C100061E043EE50E04FD20CCF82E087BB18BAC0
:100C2000EFE4F0E0808181688083EEE4F0E0808191
:100C3000896080831BBC1ABC0895EEE4F0E08081DB
:100C400081608083089590E0A0E0B0E0BC01CD0118
:100C500028D520E030E048EC52E48AD420E030E0AF
:100C60004FE753E4D4D5F1D47BBD6ABD0895E7E2E4
:100C7000F0E0808180648083E6E2F0E080818E6C29
:100C8000808308952F923F924F925F926F927F924E
:100C90008F929F92AF92BF92CF92DF92EF92FF928C
:100CA0000F931F93DF93CF93CDB7DEB72E970FB679
:100CB000F894DEBF0FBECDBF9E878D87A090B20196
:100CC000B090B301C090B401D090B501DC01509652
:100CD0002D903D904D905C90539760E070E080E8DF
:100CE0009FE3A6019501DBD33B014C01C601B50191
:100CF000ED85FE85248935894689578988D57B010C
:100D00008C01C201B101A401930181D59B01AC0109
:100D1000C801B701C5D369877A878B879C87AD8562
:100D2000BE851C968D919D910D90BC91A02D8D83BB
:100D30009E83AF83B887C601B501A201910167D533
:100D40007B018C01C401B3012D813E814F81588507
:100D50005ED59B01AC01C801B701A2D329853A85B4
:100D60004B855C859DD31B012C01ED85FE85389656
:100D7000FC83EB83C601B5012D813E814F815885EF
:100D800046D57B018C01C401B301AB81BC812D919F
:100D90003D914D915C913BD59B01AC01C801B701E0
:100DA0007FD3A20191017CD320E030E040E450E405
:100DB000DFD31B012C01ED85FE853496FA83E98390
:100DC000C601B501208131814281538120D57B014B
:100DD0008C01C401B301AD85BE852D913D914D912E
:100DE0005C9115D59B01AC01C801B70159D3EB81CA
:100DF000FC816083718382839383E090B201F090E1
:100E0000B3010091B4011091B501C801B701AD85DE
:100E1000BE852D913D914D915C91F9D45B016C01A2
:100E200060E070E080E89FE3A801970138D3A20159
:100E30009101EDD49B01AC01C601B50131D3E9812B
:100E4000FA816083718382839383AD85BE852D9201
:100E50003D924D925C9213972E960FB6F894DEBF9A
:100E60000FBECDBFCF91DF911F910F91FF90EF90FB
:100E7000DF90CF90BF90AF909F908F907F906F90BA
:100E80005F904F903F902F900895AA2797FDA095CF
:100E9000BA2FBC01CD0107D420E030E048E45DE387
:100EA000B6D40895E5E3F0E080818460808320ED8E
:100EB00037E0C9010197F1F780818B7F8083C901F9
:100EC0000197F1F70895E2E3F0E090819F77908336
:100ED00090819F7B908390819F7D908390819F7E66
:100EE0009083282F83FF03C080818068808322FF46
:100EF00005C0E2E3F0E080818064808321FF05C0CB
:100F0000E2E3F0E080818062808320FF05C0E2E3BD
:100F1000F0E08081806180830895982FE2E3F0E023
:100F200080818F77808380818F7B808380818F7D9C
:100F3000808380818F7E808399231CF480818068E8
:100F4000808396FF05C0E2E3F0E0808180648083C7
:100F500095FF05C0E2E3F0E080818062808394FF2A
:100F600005C0E2E3F0E08081806180830895FF9214
:100F70000F931F93F82EE1E3F0E08081806180837E
:100F800080818062808380818064808380818068AA
:100F90008083E5E3F0E080818160808380818D7FC4
:100FA00080838F2DBADF7EDF00ED17E0C801019747
:100FB000F1F78F2D88DF76DFC8010197F1F71F91D8
:100FC0000F91FF900895FF920F931F93F82EE1E386
:100FD000F0E0808180618083808180628083808175
:100FE0008064808380818068808305E310E0F8015D
:100FF00080818E7F808380818D7F80838F2D8DDFA8
:1010000051DFF80180818E7F80838F2D5CDF4ADF86
:101010001F910F91FF9008950F931F9320E931E0E6
:1010200048EC50E0CA010197F1F721503040D1F768
:101030008CEF82BBE5E3F0E097E0908380EF81BB2B
:1010400094BB84E0808380E368DF2CDF80E197E25B
:101050000197F1F780E361DF25DF00ED17E0C801BC
:101060000197F1F780E359DF1DDFC8010197F1F720
:1010700080E253DF17DFC8010197F1F788E2A3DFB1
:101080008CE0A1DF81E09FDF80EA9FE00197F1F72C
:1010900086E099DF1F910F910895623031F063303F
:1010A00031F0613029F4805C03C08C5E01C08C5A41
:1010B000806889DF08950F931F93CF93DF93142FD8
:1010C000052FEBDF812F902FEC01888150DF898184
:1010D00021968823D1F7DF91CF911F910F91089529
:1010E0001F93142FDADF812F42DF1F9108950F9392
:1010F0001F93082F882331F010E08EE164DF1F5F1B
:101100001017D8F31F910F9108950F931F93082F75
:10111000882331F010E088E156DF1F5F1017D8F305
:101120001F910F91089581E04EDF089582E04BDF1B
:1011300008958EE048DF08958FE045DF08958CE044
:1011400042DF089588E03FDF08958CE03CDF08959A
:101150000F931F93082F882331F010E080E133DFD5
:101160001F5F1017D8F31F910F9108950F931F93CE
:10117000082F882331F010E084E125DF1F5F10176E
:10118000D8F31F910F910895EF92FF920F931F9341
:10119000CF93DF93182F062FEA01CA0168EE73E0A0
:1011A00099D3862F972F009731F0462F405D812FDE
:1011B000602F96DF04C0812F602F40E391DFCE01C6
:1011C00068EE73E087D3F82EE92E64E670E082D3F0
:1011D000862F972F009739F0462F405D812F8F5F24
:1011E000602F7EDF05C0812F8F5F602F40E378DFA7
:1011F0008F2D9E2D64E670E06DD3F82EE92E6AE007
:1012000070E068D3862F972F009739F0462F405D06
:10121000812F8E5F602F64DF05C0812F8E5F602F6E
:1012200040E35EDF8F2D9E2D6AE070E053D3009780
:1012300039F0482F405D812F8D5F602F51DF05C051
:10124000812F8D5F602F40E34BDFDF91CF911F91A6
:101250000F91FF90EF9008956F927F928F929F92DF
:10126000AF92BF92CF92DF92EF92FF920F931F93B4
:10127000CF93DF93D62EC72EB82EA92E842E922E72
:10128000380120E030E040E050E06ED188231CF0CF
:10129000C0E0D0E005C08DE28093B601C1E0D0E0AF
:1012A000E92CFF24E114F10439F48D2D9C2DAB2D94
:1012B000BA2DBC01CD0112C08D2D9C2DAB2DBA2DA8
:1012C000BC01CD0100E010E020E030E040E251E45C
:1012D0009ED20F5F1F4F0E151F05B0F320E030E0C8
:1012E00040E05FE3DDD0ACD1DC01CB018C0160E1FB
:1012F00077E2F0D2862F972F009731F0FE01EA5463
:10130000FE4F805D80832196C80160E177E2E2D2E2
:10131000482F192F68EE73E0DDD2862F972F0097A4
:1013200039F0FE01EA54FE4F805D8083219610C0A3
:10133000209771F0FE01EB54FE4FE081E13340F065
:10134000EA3330F4FE01EA54FE4F80E380832196B5
:10135000842F912F68EE73E0BDD2482F192F64E6D9
:1013600070E0B8D2862F972F009739F0FE01EA542B
:10137000FE4F805D8083219610C0209771F0FE01A2
:10138000EB54FE4FE081E13340F0EA3330F4FE01EC
:10139000EA54FE4F80E380832196842F912F64E6E8
:1013A00070E098D2482F192F6AE070E093D2862F10
:1013B000972F009739F0FE01EA54FE4F805D80833D
:1013C000219606C0FE01EA54FE4F80E380832196F9
:1013D000842F912F6AE070E07DD2009741F0FE01EA
:1013E000EA54FE4F805D8083FE01319607C0FE0106
:1013F000EA54FE4F80E38083FE013196482D50E091
:10140000BF014E175F0708F4BA01FB01EA54FE4F13
:1014100010826115710519F420E030E027C040E02A
:1014200050E020E030E0CB018E199F097C010EE2F4
:1014300012E09EE2C6EBD1E0992049F0E416F506F1
:1014400031F4F801E20FF31F90832F5F3F4FF80153
:10145000E20FF31FDE01A40FB51F8C9180832F5F75
:101460003F4F4F5F5F4F4617570730F36EE272E012
:10147000FB01E20FF31F1082F3011082C3013ED281
:10148000DF91CF911F910F91FF90EF90DF90CF9060
:10149000BF90AF909F908F907F906F90089550581D
:1014A000BB27AA270ED075C166D130F06BD120F0D2
:1014B00031F49F3F11F41EF45BC10EF4E095E7FB9D
:1014C00051C1E92F77D180F3BA17620773078407F8
:1014D000950718F071F49EF58FC10EF4E0950B2E70
:1014E000BA2FA02D0B01B90190010C01CA01A00176
:1014F0001124FF27591B99F0593F50F4503E68F1D1
:101500001A16F040A22F232F342F4427585FF3CF11
:10151000469537952795A795F0405395C9F77EF4E2
:101520001F16BA0B620B730B840BBAF09150A1F02B
:10153000FF0FBB1F661F771F881FC2F70EC0BA0FB1
:10154000621F731F841F48F4879577956795B79539
:10155000F7959E3F08F0B3CF9395880F08F0992731
:10156000EE0F979587950895D9D008F481E00895F6
:101570000CD00FC107D140F0FED030F021F45F3F16
:1015800019F0F0C0511139C1F3C014D198F3992367
:10159000C9F35523B1F3951B550BBB27AA27621737
:1015A0007307840738F09F5F5F4F220F331F441F7C
:1015B000AA1FA9F333D00E2E3AF0E0E830D09150B4
:1015C0005040E695001CCAF729D0FE2F27D0660FA1
:1015D000771F881FBB1F261737074807AB07B0E8E0
:1015E00009F0BB0B802DBF01FF2793585F4F2AF0F6
:1015F0009E3F510568F0B6C000C15F3FECF3983ED6
:10160000DCF3869577956795B795F7959F5FC9F752
:10161000880F911D9695879597F90895E1E0660FDB
:10162000771F881FBB1F621773078407BA0720F054
:10163000621B730B840BBA0BEE1F88F7E0950895BD
:1016400004D06894B111D9C00895BCD088F09F57D8
:1016500090F0B92F9927B751A0F0D1F0660F771FFE
:10166000881F991F1AF0BA95C9F712C0B13081F0DE
:10167000C3D0B1E00895C0C0672F782F8827B85F26
:1016800039F0B93FCCF3869577956795B395D9F73F
:101690003EF490958095709561957F4F8F4F9F4F49
:1016A0000895E89409C097FB3EF490958095709555
:1016B00061957F4F8F4F9F4F9923A9F0F92F96E99E
:1016C000BB279395F695879577956795B795F11113
:1016D000F8CFFAF4BB0F11F460FF1BC06F5F7F4FB0
:1016E0008F4F9F4F16C0882311F096E911C07723C2
:1016F00021F09EE8872F762F05C0662371F096E8CB
:10170000862F70E060E02AF09A95660F771F881F99
:10171000DAF7880F9695879597F90895990F00083D
:10172000550FAA0BE0E8FEEF16161706E807F907B3
:10173000C0F012161306E407F50798F0621B730B4E
:10174000840B950B39F40A2661F0232B242B252BCF
:1017500021F408950A2609F4A140A6958FEF811D72
:10176000811D089597F99F6780E870E060E0089513
:101770009FEF80EC089500240A94161617061806A9
:101780000906089500240A94121613061406050685
:101790000895092E0394000C11F4882352F0BB0F16
:1017A00040F4BF2B11F460FF04C06F5F7F4F8F4F79
:1017B0009F4F089557FD9058440F551F59F05F3FB4
:1017C00071F04795880F97FB991F61F09F3F79F063
:1017D00087950895121613061406551FF2CF4695E5
:1017E000F1DF08C0161617061806991FF1CF869567
:1017F0007105610508940895E894BB27662777274B
:10180000CB0197F908958ADF08F48FEF08950BD084
:10181000C0CFB1DF28F0B6DF18F0952309F0A2CFD2
:10182000A7CF1124EACFC6DFA0F3959FD1F3950F80
:1018300050E0551F629FF001729FBB27F00DB11D54
:10184000639FAA27F00DB11DAA1F649F6627B00DE4
:10185000A11D661F829F2227B00DA11D621F739FCD
:10186000B00DA11D621F839FA00D611D221F749FDB
:101870003327A00D611D231F849F600D211D822F22
:10188000762F6A2F11249F5750408AF0E1F0882369
:101890004AF0EE0FFF1FBB1F661F771F881F915076
:1018A0005040A9F79E3F510570F05CCFA6CF5F3F37
:1018B000ECF3983EDCF3869577956795B795F795A9
:1018C000E7959F5FC1F7FE2B880F911D9695879531
:1018D00097F90895AA1BBB1B51E107C0AA1FBB1FA4
:1018E000A617B70710F0A61BB70B881F991F5A95AC
:1018F000A9F780959095BC01CD010895FB01DC010D
:1019000001900D920020E1F70895FB01DC010D909C
:101910000020E9F711974150504028F00190002035
:0E1920000D92C9F708951C920895F894FFCF18
:10192E005A72004F7600467300587A004C65616417
:10193E0020416369642042617474727900202D2DF8
:10194E002D2D2D2D2D2D2D2D2D2D2D2D2D005642A8
:10195E0000546F6F204C4F572056483D20202020BA
:10196E0020004E6F20424154542056423D202020EC
:10197E0020202000446574656374696E6720534FA0
:10198E00432E2E2E00446574656374656420534F98
:10199E00433D20202000483D00423D004100643D73
:1019AE000025002D2D2D204E6F20416374696F6E22
:1019BE00202D2D004C4142204368617267657220D4
:1019CE00332E304500537570706C7920004261746F
:1019DE007465727920004D4F534645542000566F62
:1019EE006C743A2000437572723A2000546172672B
:1019FE0065742000447574793A200020562C20001E
:101A0E0020412C200020252C20000A000000000080
:101A1E00000000000000000000000000000000CDEB
:101A2E00CCCC3D0501000000000034332341000002
:101A3E006441000070417500770079007B007C00E6
:101A4E007D007E007F007F007F0075007C007F00A0
:101A5E008100820083008400850088008D000A00CA
:101A6E0014001E00280032003C00460050005A00B0
:0E1A7E0064006666263F2020202020202020C5
:00000001FF
